:100000000C9456000C9468000C9468000C946800E2
:100010000C9468000C9468000C9468000C946800C0
:100020000C9468000C9468000C9468000C946800B0
:100030000C9468000C9468000C9468000C946800A0
:100040000C9468000C9468000C9468000C94680090
:100050000C9468000C9468000C9468000C94680080
:100060000C9468000C9468000C9468000C94680070
:100070000C9468000C9468000C9468000C94680060
:100080000C9468000C9468000C9468000C94680050
:100090000C9468000C9468000C9468000C94680040
:1000A0000C9468000C9468000C94680011241FBE26
:1000B000CFEFCDBFD7E2DEBF20E2A0E0B0E201C0CB
:1000C0001D92AC31B207E1F70E946A010C94A001C5
:1000D0000C940000DC01FA0110828C918623E9F770
:1000E0008DE28A95F1F700008AE58A95F1F700C064
:1000F0008C91862319F08081816080838AE58A95BE
:10010000F1F700C08C91862319F080818260808392
:100110008AE58A95F1F700C08C91862319F08081D9
:10012000846080838AE58A95F1F700C08C918623EC
:1001300019F08081886080838AE58A95F1F700C094
:100140008C91862319F08081806180838AE58A956D
:10015000F1F700C08C91862319F080818062808342
:100160008AE58A95F1F700C08C91862319F0808189
:10017000806480838AE58A95F1F700C08C9186239C
:1001800019F08081806880838AE58A95F1F700C044
:100190008DE28A95F1F700000895FC019081862F89
:1001A0008095982390839AE59A95F1F700C0908105
:1001B00040FF02C0962B01C0982390839AE59A9540
:1001C000F1F700C0908141FF02C0962B01C0982337
:1001D00090839AE59A95F1F700C0908142FF02C0A2
:1001E000962B01C0982390839AE59A95F1F700C069
:1001F000908143FF02C0962B01C0982390839AE51B
:100200009A95F1F700C0908144FF02C0962B01C07F
:10021000982390839AE59A95F1F700C0908145FF65
:1002200002C0962B01C0982390839AE59A95F1F726
:1002300000C0908146FF02C0962B01C09823908396
:100240009AE59A95F1F700C047FF04C08081862B9C
:10025000808303C09081982390838AE58A95F1F783
:1002600000C08081862B80839AE59A95F1F700C0C3
:100270008AE58A95F1F700C00895FF920F931F93C6
:10028000CF93DF938C01F62EEA0110921A20109280
:100290001B20E0911A20F0911B20EC0FFD1F4081E4
:1002A0006F2DC8010E94CD0020911A2030911B2093
:1002B0002F5F3F4F20931A2030931B20FE01E20F47
:1002C000F31F80818111E5CFDF91CF911F910F91B5
:1002D000FF90089582E0809350008091510081FF4B
:1002E000FCCF88ED84BF81E080934000CF9AC79A0D
:1002F000849A00E010E049E150E260E48AE190E095
:100300000E946A008C9AE8012196F801E050F04EB4
:100310008C2F805D8083C831D10511F4C0E0D0E01E
:1003200040E050E260E889E190E00E943D014AE04F
:1003300060E889E190E00E94CD008C988E01DBCFCF
:04034000F894FFCF5F
:00000001FF
